:10000000182AFF3FFF3FFF3FCF00030E8301A400EC
:100010000408A5000A08A6008A014108AC004008AF
:10002000AB000B1D41290030861B0130C200420885
:100030000130031D0030C3000030061B0130C20038
:1000400042080130031D0030C0004308C0050C0801
:10005000C005003040188030060680398606013021
:100060000505C0000D08C006C1010030C1064008EA
:10007000410403195C288E0A03198F0A11086D3C8C
:10008000031D44281008603C0318592892011308E6
:100090000319542815089400170896000330980097
:1000A00099019A0101309B00950197019C019301F0
:1000B0000515900191011629900A0319910A0F085C
:1000C000003C031D65280E08003C031814290F0886
:1000D0000A3C031D6D280E08F03C0318DB28013094
:1000E0009D009728970ACB2802309707CB28043029
:1000F0009707CB2808309707CB280A309707CB28DB
:1001000014309707CB2828309707CB28950ACB289F
:1001100002309507CB2804309507CB280830950787
:10012000CB280A309507CB2814309507CB28120826
:10013000153A031972281208163A0319742812087E
:10014000173A031977281208183A03197A2812085F
:10015000193A03197D2812081A3A0319802812083F
:100160001B3A0319832812081D3A0319862812081E
:100170001E3A0319882812081F3A03198B281208FF
:10018000203A03198E281208213A031991281208DF
:10019000223A0319942812081C3A0319D928120884
:1001A000233A0319D92812083A3A0319D928D8282A
:1001B0009C0A920AF3280F08053C031DE1280E084B
:1001C000783C0318EF281208143A031DEC28FF307E
:1001D0009D0092010511EE289D01920AF328FF303F
:1001E0009D00920105111208153A031DF8289C0183
:1001F00012081D3A031905291208243A0319052982
:1002000012083B3A031905290F2901301C05C200C9
:1002100042081D0603190E29920105119C011208BE
:100220003B3A031D1429930A8E018F01990A031981
:100230009A0A1A084C3C031D1F2919084B3C031845
:10024000352999019A01980A18083C3A031D352965
:100250009801960A16083C3A031D35299601940A1E
:100260001408183A031D3529940101300505C00012
:100270000D08C00600304018023005060239850618
:100280000B112C08C1002B08C00026088A00250885
:100290008400240E8300CF0E4F0E09000313831237
:1002A0002A0803196529A230CB00FF30CA00CB0B06
:1002B0005A295D29CA0B5A295729EA30CA00CA0BA4
:1002C0005F2900000000AA034E29080003138312CF
:1002D000C8010830CC00400DC80D4408C8020318FE
:1002E0007329C8070310C00DCC0B6B29080003133A
:1002F00083122708890083168813081483120808BC
:10030000C00008000130031383128C00A701A8016C
:1003100028081E02031CB529A9010A302902031866
:10032000B329280886000130AA004E211F0828069C
:10033000031D9D290F30C0009F292808C0004008D8
:1003400086000130AA004E21851DB1290F3086009C
:100350000830AA004E21280886008C012808A00039
:100360000800A90A8D29A80A88290A301F02031843
:10037000C229A70A2708033A031DC2298C011F08B6
:10038000A000080087290800000003138316881CBA
:10039000CB290000C5292708831289002808880076
:1003A0008316881308158B1355308900AA308900ED
:1003B00088148B17081108000F300313831286006E
:1003C0000A30AA004E210A30C4002708C000662166
:1003D000400886001030AA004E210F3086000230FF
:1003E000AA004E210A30C4002708C0006621480830
:1003F000C000400886000C30AA004E2108000313FC
:1004000083124008C100C0010830CC004108C40C70
:1004100003180E2ACC0B072AC10100340310132A3B
:10042000C40C0318C107C10CC00CCC0B102A080067
:10043000093003138316850040308600A0308B00FE
:10044000D83081009B01A701772140089F0002302E
:100450009E0082210313831220088D000A309F0022
:100460002008023A031D5E2A02309E0082210313F7
:1004700083122008C0000A30C400FF214008940005
:1004800009309E008221031383122008940705304F
:100490009E008221031383122008C0000A30C4008A
:1004A000FF214008960009309E0082210313831229
:1004B000200896070330980001309B000313831235
:1004C000A7010D08A800C421031383121B08003CD8
:1004D0000318BF2A851D8E2AA10118300313831229
:1004E000210203188D2A01308C002108A700DC218D
:1004F0002108103FA700772140089F0001309E008F
:100500008221031383122108103FA7002008A800AE
:10051000C42103138312A10A6D2ABF2A0F300313CB
:100520008312860001308C000130AA004E21180889
:10053000A2001608A3001408A1001408A700DC21DB
:100540002308A700DC212208A700DC218C01210858
:10055000103FA700772140080319B22A3C30AA00B7
:100560004E21BF2A031383120D08023A031DBC2A31
:10057000FF30AA004E21BF2A031383129B01642A75
:10058000C02AFF3FFF3FFF3FFF3FFF3FFF3FFF3FCF
:104200000100FF00FF00FF00FF00FF00FF00FF00B4
:10421000FF00FF00FF00FF00FF00FF00FF00FF00A6
:104220000100010001000100010001000100010086
:104230000100010001000100010001000100010076
:104240000100010001000100010001000100010066
:10425000FF00FF00FF00FF00FF00FF00FF00FF0066
:10426000FF00FF00FF00FF00FF00FF00FF00FF0056
:10427000FF00FF00FF00FF00FF00FF00FF00FF0046
:10428000FF00FF00FF00FF00FF00FF00FF00FF0036
:10429000FF00FF00FF00FF00FF00FF00FF00FF0026
:1042A000FF00FF00FF00FF00FF00FF00FF00FF0016
:1042B000FF00FF00FF00FF00FF00FF00FF00FF0006
:1042C000FF00FF00FF00FF00FF00FF00FF00FF00F6
:1042D000FF00FF00FF00FF00FF00FF00FF00FF00E6
:1042E000FF00FF00FF00FF00FF00FF00FF00FF00D6
:1042F000FF00FF00FF00FF00FF00FF00FF00FF00C6
:10430000FF00FF00FF00FF00FF00FF00FF00FF00B5
:10431000FF00FF00FF00FF00FF00FF00FF00FF00A5
:10432000FF00FF00FF00FF00FF00FF00FF00FF0095
:10433000FF00FF00FF00FF00FF00FF00FF00FF0085
:10434000FF00FF00FF00FF00FF00FF00FF00FF0075
:10435000FF00FF00FF00FF00FF00FF00FF00FF0065
:10436000FF00FF00FF00FF00FF00FF00FF00FF0055
:10437000FF00FF00FF00FF00FF00FF00FF00FF0045
:10438000FF00FF00FF00FF00FF00FF00FF00FF0035
:10439000FF00FF00FF00FF00FF00FF00FF00FF0025
:1043A000FF00FF00FF00FF00FF00FF00FF00FF0015
:1043B000FF00FF00FF00FF00FF00FF00FF00FF0005
:1043C000FF00FF00FF00FF00FF00FF00FF00FF00F5
:1043D000FF00FF00FF00FF00FF00FF00FF00FF00E5
:1043E000FF00FF00FF00FF00FF00FF00FF00FF00D5
:1043F000FF00FF00FF00FF00FF00FF00FF00FF00C5
:02400E00FA3F77
:00000001FF
